:100000000C9446000C9463000C9463000C94630001
:100010000C9463000C9463000C9463000C946300D4
:100020000C9463000C9463000C9463000C946300C4
:100030000C9463000C9463000C9463000C946300B4
:100040000C9463000C9463000C9463000C946300A4
:100050000C9463000C9463000C9463000C94630094
:100060000C9463000C9463000C9463000C94630084
:100070000C9463000C9463000C9463000C94630074
:100080000C9463000C9463000C94630011241FBE55
:10009000CFEFD0E1DEBFCDBF11E0A0E0B1E0E4EDF5
:1000A000F1E000E00BBF02C007900D92A633B1074C
:1000B000D9F711E0A6E3B1E001C01D92A833B10762
:1000C000E1F70C949A000C9400009C0144275527FA
:1000D000220F331F441F551F220F331F441F551F6C
:1000E000220F331F441F551F220F331F441F551F5C
:1000F00060E070E081EE90E00E94AD002150304061
:10010000832F9927809398002093990088E080930B
:100110009A000895882321F45D9BFECF6CB9089561
:10012000813039F4EBE9F0E0808185FFFDCF609309
:100130009C000895CFEFD0E1DEBFCDBF80E895E20F
:100140000E946500C0E0D1E0699181E00E948A00D0
:1001500081E0C633D807C1F7FFCF97FB092E0526EC
:100160000ED057FD04D014D00AD0001C38F450959E
:100170004095309521953F4F4F4F5F4F0895F6F7CB
:1001800090958095709561957F4F8F4F9F4F089503
:10019000A1E21A2EAA1BBB1BFD010DC0AA1FBB1F8B
:1001A000EE1FFF1FA217B307E407F50720F0A21BFD
:1001B000B30BE40BF50B661F771F881F991F1A946A
:1001C00069F760957095809590959B01AC01BD0194
:0401D000CF010895BE
:1001D40091839104C3888C05C0A205A98605AA80D1
:1001E40000AE80008C9BC29489058C9AA69481C22F
:1001F40005BBC680C204A583BF05BF83BBBF05C7BB
:060204009489B394848C80
:00000001FF
